:020000000F28C7
:080008000B110900F6000030A5
:100010008A000F30760703188A0A76088207203094
:1000200083120313BB000430BC000230BD00D701B3
:1000300083120313D8010930D9000230DA000130ED
:10004000DB000230DC000830DD000330DE0004306D
:100050008600F03083168500F23086004030810043
:100060008B01EE260730831203139F00193083168D
:100070009900243098009030831298008C01B701C9
:100080000130B600B901B8013030CA006427B701A9
:100090000230B600B901B8014030CA006427FA3016
:1000A000B400A127FA30B400A127FA30B400A12788
:1000B0002B2783120313B7010230B600B901B80130
:1000C000CA016427F724F724831203130608F000FB
:1000D000F00CF00CF00C700C0F39F0007008063CBE
:1000E000031D7C2883120313A001A101A201A30117
:1000F0008F30A400DC24F6297008073C031DDF289C
:100100000130831203135B02031DB6280530580229
:10011000013003180301F1005808073C01300318AF
:1001200003017104003C0319AF285808093C013051
:1001300003190301F10058080B3C013003190301B6
:100140007105003C0319AF285808A000A101A201C5
:10015000A3010730A400DC2483120313CC00D80AC7
:100160000D305802031DF629D801F62902308312FA
:1001700003135B02031DC52806305E02031DC3285E
:100180000130DE00DE28DE0ADE280330831203138E
:100190005B02031DDE28A001A101A201A3015D08ED
:1001A000A400DC2483120313CC0008305D02031D7D
:1001B000DC288830DD00DE280830DD00F6297008F4
:1001C0000B3C031D64290130831203135B02031DE2
:1001D000422901305002031D0929F1015508103E42
:1001E0000318F10AD500F100F10CF10CF10C710CBF
:1001F0000F390E3C031D24295508F100710EF0390A
:10020000F039F100F10CF10CF10C710C0F39D50043
:100210002429F101831203135508013E0318F10A42
:10022000D500F100710EF039F039E03C031D2429AE
:100230005508F100F10CF10CF10C710C0F39F100C3
:10024000710EF039F039D500CB01BF275930831238
:100250000313CB00BF27831203135508CB00BF271E
:10026000831203135608CB00BF27BC30831203133D
:10027000CB00BF27CE2783120313CC000A30B40073
:10028000A127F62902305B02031D4B29C2015E083B
:10029000C300372563290330831203135B02031D58
:1002A0006329A001A101A201A3015C08A400DC2430
:1002B00083120313CC00CC08031D61298230DC00BB
:1002C00063290230DC00F62970080D3C031DB129BA
:1002D0000130831203135B02031D7929A001A101E0
:1002E000A201A3018130A400DC2483120313CC00FB
:1002F000F62902305B02031D83290130C2005E082B
:10030000C3003725B0290330831203135B02031D9A
:10031000B02954080C3C0130031D0301F1005408BE
:10032000C03C0130031D03017104003C0319B029D6
:100330005908A000A101A201A3010930A400DC24F6
:1003400083120313CC0089305902031DAA290930F6
:10035000D900B029F1015908403E0318F10AD9002B
:10036000F62970080E3C031DF6290430831203138E
:100370005A02031DBD290130DA003230B400A12732
:100380005A08F1007108013C031DD229831203139E
:10039000B7010230B600B901B801CA0164270130C3
:1003A000DB00F4297108023C031DE32983120313C7
:1003B000B7010230B600B901B8011030CA00642795
:1003C0000230DB00F4297108033C031DF429831279
:1003D0000313B7010230B600B901B8012030CA00DA
:1003E00064270330DB00F429DA0AF629F724CB016D
:1003F000BF27593083120313CB00BF278312031387
:10040000CB01BF2783120313CB01BF27BB3083125D
:100410000313CB00BF27CE2783120313D500CE27AB
:1004200083120313D600CB01BF2755308312031369
:10043000CB00BF2783120313CB01BF278312031303
:10044000CB01BF27BB3083120313CB00BF27CE27BE
:10045000FE00CE27FF007E088039003C03196C2A7D
:100460007E08F0007008813C031D3D2A4230831253
:100470000313D3000130D000772A7008803C031D9D
:10048000472A413083120313D300D001772A700822
:10049000903C031D4C2A502A7008913C031D532A9E
:1004A0004830D300772A7008843C031D582A5C2A00
:1004B0007008853C031D5F2A5130D300772A7008ED
:1004C000863C031D642A682A7008873C031D6B2A3A
:1004D0007430D300772A772A4D3083120313D30068
:1004E0007E082039003C0319772A5430D3000130AC
:1004F000BF00C0015308C1002925F0013030F100D0
:10050000831203132508F200F20CF20CF20C720CA9
:100510000F3971070318F00AAA00303C031D922A14
:100520002030AA00F0013030F1002508F200720EF0
:10053000F039F039F200F20CF20CF20C720C0F39B7
:1005400071070318F00AAB002A08203C0130031D94
:100550000301F0002B08303C0130031D030170053E
:10056000003C0319B52A2030AB00F0013030F10017
:100570002608F200F20CF20CF20C720C0F39710723
:100580000318F00AAC002E30AD00F0013030F1005D
:100590002608F200720EF039F039F200F20CF20C7B
:1005A000F20C720C0F3971070318F00AAE00F0015B
:1005B0003030F1002708F200F20CF20CF20C720C51
:1005C0000F3971070318F00AAF00F0013030F10065
:1005D0002708F200720EF039F039F200F20CF20C3A
:1005E000F20C720C0F3971070318F00AB0002E30AC
:1005F000B100F0013030F1002808F200F20CF20CEA
:10060000F20C720C0F3971070318F00AB200F001F6
:100610003030F1002808F200720EF039F039F200A3
:10062000F20CF20CF20C720C0F3971070318F00A7D
:10063000B3005708093C031C322B0130BF00F00106
:10064000023057070318F00AC00057082A3E8400FA
:100650008313000883120313C10029258312031397
:10066000D70A192BD7015708023C031C5B2B01301A
:10067000BF00F0010D3057070318F00AC000290829
:10068000F7000330F800EA27F0007808583EF10040
:100690000318F00A7108831203135707F1000318B7
:1006A000F00A7108BE0021258312C100292583129A
:1006B0000313D70A332BD70101305002031D6D2BD2
:1006C0000330D1003C30D2005508F000F00CF00CA3
:1006D000F00C700C0F39D400772B0130D100B630FC
:1006E000D2005508F000700EF039F039D4005408EB
:1006F0000C3C0130031D0301F0005408C03C0130E4
:10070000031D03017004003C0319B42B5108CB00F6
:10071000BF27831203135208CB00BF278312031392
:10072000CB01BF2783120313CB01BF27BB3083123A
:100730000313CB00BF27CE27FE00CE27FF007E0885
:10074000643C031DA82B2D3083120313D300B82B58
:100750007E08A43C031DB12B2B3083120313D3005E
:10076000B32B2030D300B82B203083120313D300D7
:100770000130BF000C30C0005308C100292583128E
:100780000313CB01BF27793083120313CB00BF279C
:1007900083120313CB01BF2783120313CB01BF279F
:1007A000BB3083120313CB00BF27CE27FE00CE271A
:1007B000FF007E08F000700EF039F039F00070088C
:1007C000003C031DE42BE82B7008403C031DED2B7F
:1007D000343083120313D300132C7008103C031D14
:1007E000F22BF62B7008503C031DFB2B3330831289
:1007F0000313D300132C7008203C031D002C042C81
:100800007008603C031D072C3230D300132C700895
:10081000303C031D0C2C102C7008703C031D132C55
:100820003130D300132C0230BF000530C000530814
:10083000C10029257F088039003C03192D2C033085
:10084000831203135B02031D362C0230BF000C30F1
:10085000C0002A30C1002925362C02308312031330
:10086000BF000C30C0002030C100292583120313C3
:10087000A001A101A201A301F730A400DC2483128E
:100880000313CC008039031D612C0230BF00C0016E
:100890005030C1002925831203134C1F572C0230FE
:1008A000BF000330C0004830C10029257E2C023033
:1008B00083120313BF000330C0004C30C100292550
:1008C0007E2C023083120313BF00C0017330C100BD
:1008D000292583120313A001A101A201A301E7307E
:1008E000A400DC2483120313CC008039031D7E2C6A
:1008F0000230BF00C0015330C10029258312031309
:100900004C08F000700EF039F039F000F00CF00CEB
:10091000F00C700C0F39CD0001304D02031CAD2CD2
:1009200001304D020130031C0301F0004D08093C69
:100930000130031C03017005003C0319A82CF001D1
:1009400030304D070318F00ACE002030CF00B22C13
:100950003930CE002B30CF00B22C2030831203135D
:10096000CE00CF000230BF000130C0004E08C100F1
:100970002925023083120313BF00C0004F08C100B5
:1009800029250230831203135B02031DD22C02308F
:10099000BF000F30C000F00130305E070318F00ACE
:1009A000C1002925023083120313BF000630C000A6
:1009B0007C30C10029256428831203132008CB0052
:1009C000BF27831203132108CB00BF278312031311
:1009D0002208CB00BF27831203132308CB00BF27B5
:1009E000831203132408CB00BF27CE2708008312ED
:1009F0000313CB01BF2783120313CB01BF2783123D
:100A00000313CB01BF2783120313CB01BF2703308E
:100A100083120313CB00BF27CE2783120313A50035
:100A2000CE2783120313A600CE2783120313A70039
:100A3000CE2783120313A800CE2783120313A90025
:100A40000800831203133E0883169B001C141A0827
:100A50000800831203133F08C8004008C900372765
:100A60008312031306144108C7001427080030300E
:100A700083120313E1003930E2004208003C0319FD
:100A8000462D6208DF006108E0004A2D6108DF00A2
:100A90006208E0004308063C031C7E2E33085F0218
:100AA0000130031D0301F100023043020130031C39
:100AB0000301F2004308063C0130031C03017205E8
:100AC0007104003C0319732E01304302031D6A2D8B
:100AD0006008B30032085F020130031D0301F1001A
:100AE000033043020130031C0301F2004308063CBB
:100AF0000130031C030172057104003C0319682EC8
:100B00004308013C0130031D0301F1004308023C8E
:100B10000130031D03017104003C0319912D60088D
:100B2000B20030085F020130031D0301F100043000
:100B300043020130031C0301F2004308063C01306C
:100B4000031C030172057104003C0319562E013089
:100B500043020130031C0301F1004308033C013050
:100B6000031C03017105003C0319B82D6008B00097
:100B70002F085F020130031D0301F100053043021D
:100B80000130031C0301F2004308063C0130031C42
:100B9000030172057104003C03194B2E013043021E
:100BA0000130031C0301F1004308043C0130031C25
:100BB00003017105003C0319DF2D6008AF002E080A
:100BC0005F020130031D0301F1004308063C0130C0
:100BD000031D03017104003C0319402E0130430240
:100BE0000130031C0301F1004308053C0130031CE4
:100BF00003017105003C0319FF2D6008AE002C08AD
:100C00005F02031D352E013043020130031C030136
:100C1000F1004308063C0130031C03017105003C50
:100C20000319142E6008AC002B085F02031D2A2E46
:100C30006008AB002A085F02031D212E6008AA008D
:100C40007E2E2A08C4004208C5000130C600DC26FA
:100C5000AA007E2E831203132B08C4004208C5008D
:100C60000130C600DC26AB007E2E831203132C0855
:100C7000C4004208C5000130C600DC26AC007E2E50
:100C8000831203132E08C4004208C5000130C600B9
:100C9000DC26AE007E2E831203132F08C400420808
:100CA000C5000130C600DC26AF007E2E8312031380
:100CB0003008C4004208C5000130C600DC26B00080
:100CC00003304302031D672E3030B200B3007E2E86
:100CD000831203133208C4004208C5000130C60065
:100CE000DC26B2007E2E831203133308C4004208B0
:100CF000C5000130C600DC26B3007E2EF101831250
:100D000003132A08F200720EF039F039F2002B08B2
:100D1000F300730EF039F039F300F30CF30CF30C1D
:100D2000730C0F3972070318F10AA000F1012C08A7
:100D3000F200720EF039F039F2002E08F300730E53
:100D4000F039F039F300F30CF30CF30C730C0F399A
:100D500072070318F10AA100F1012F08F200720EC8
:100D6000F039F039F2003008F300730EF039F03941
:100D7000F300F30CF30CF30C730C0F397207031828
:100D8000F10AA200F1013208F200720EF039F039D6
:100D9000F2003308F300730EF039F039F300F30C6E
:100DA000F30CF30C730C0F3972070318F10AA3004C
:100DB0000130A400DC240800831203134508003C22
:100DC0000319E92EF101440846070318F10AC4008B
:100DD000EC2E46084402C4004408080083120313A2
:100DE000861106100530B400A127033085002627A0
:100DF0000530B400A1270230850026270530B40055
:100E0000A1272830C7001427083083120313C70016
:100E100014270C3083120313C700142706308312E3
:100E20000313C70014270800831203134708F300B5
:100E3000F30CF30CF30C730C0F39850026274708CD
:100E4000850026272830BA00B22708008312031332
:100E50008615861108008312031306100130C7009F
:100E60001427023083120313B400A1270800831251
:100E7000031306104808F2007208013C031D4A2FB4
:100E8000F30180308312031349070318F30AC700E4
:100E900014275E2F7208023C031D5E2FF3014030C1
:100EA0008312031349070318F30AF4007308003888
:100EB000F30074088038C70014275E2F02308312B5
:100EC0000313B400A127080083120313DF01E0011C
:100ED0006008003C0030031C752F0130031D752F86
:100EE0005F080F3C0130031C0301003C0319A02FD5
:100EF0003708F2003608C8003908F2006008F20727
:100F000038085F070318F20AC90037278312031352
:100F100006140030F2006008F2074A085F07031861
:100F2000F20ABE002125013CF2007209013E831243
:100F3000C700142783120313DF0A0319E00A682F7E
:100F400008008E3083120313B5000000000000007B
:100F5000000000000000B50BA72F0000B40BA12F6C
:100F60000000080083120313BA0CBA0C3F30BA0514
:100F70000330BA020000BA0BBA2F00000800831237
:100F800003134B08990083168312031301080319F6
:100F9000CC2F83161808C42F831208008312031362
:100FA0000C083B05FF39003C0319CE2F18083C05FF
:100FB000FF39F10018083D05FF397104003C0319A1
:100FC000E62F1812000018161A08E3001A08080085
:100FD000CE2F08000930F9007708F7010310F70C4D
:0E0FE000F80C0318F707F90BEF2F770808003D
:02400E00503F21
:104200002100210021002100210021002100570070
:10421000670021004300650021004E006500210079
:104220002100210021002100210021002100560051
:104230007100210045007800210054007500210024
:104240002100210021002100210021002100530034
:10425000710021005400710021005100550021001F
:10426000470055002E00390032003800210053006D
:1042700066006E007000750066004E0062006F0000
:104280004A00580033004D004700450021007300EC
:1042900032002F003300210033003100310036009E
:1042A00020002000720031002E0032002E0032006B
:1042B0004C005300420055005300420020004300D0
:1042C0005700430057005200200041004D000000FD
:1042D00000000000570046004D00000000000000F4
:1042E000200046004D00000000000000440049008E
:1042F000470000000000000050004B005400000088
:00000001FF
